:020000021000EC
:10F800000C9446FC0C9463FC0C9463FC0C9463FC19
:10F810000C9463FC0C9463FC0C9463FC0C9463FCEC
:10F820000C9463FC0C9463FC0C9463FC0C9463FCDC
:10F830000C9463FC0C9463FC0C9463FC0C9463FCCC
:10F840000C9463FC0C9463FC0C9463FC0C9463FCBC
:10F850000C9463FC0C9463FC0C9463FC0C9463FCAC
:10F860000C9463FC0C9463FC0C9463FC0C9463FC9C
:10F870000C9463FC0C9463FC0C9463FC0C9463FC8C
:10F880000C9463FC0C9463FC0C9463FC11241FBE69
:10F89000CFEFD0E1DEBFCDBF11E0A0E0B1E0ECECF6
:10F8A000FFEF01E00BBF02C007900D92A030B1073F
:10F8B000D9F712E0A0E0B1E001C01D92A434B10775
:10F8C000E1F70C94AAFF0C9400FC0F93EF93FF93C5
:10F8D00040D0FC01062F36D0FF91EF910F91089593
:10F8E0000F930F921F92EF93FF9333D0FC010B0104
:10F8F00001E028D0FF91EF911F900F900F91089594
:10F900000F930F92EF93FF9324D0FC0160FD60935F
:10F910006800D895802DE395D895902DFF91EF91B3
:10F920000F900F9108950F930F9213D0082E09E0B6
:10F9300009D00F900F9108950F930BD001E102D0E1
:10F940000F910895E199FECF00936800E895FFFFBD
:10F9500000000091680000FDFCCF089583E089B9A4
:10F96000549A539A08958CB19927089540E050E035
:10F970004817590750F42AE633E000002150304080
:10F9800037FFFBCF4F5F5F4FF3CF08958BB19927C0
:10F990008078907008955498539808950E94CBFCF5
:10F9A0000C94000008958CB95E9BFECF5E9A08957A
:10F9B0000E94C6FC8823E1F30E94B3FC803219F454
:10F9C00081E090E0089585E10E94D3FC80E090E022
:10F9D00008950895EF92FF920F931F93CF93DF93B3
:10F9E0007B01C0E0D0E0C617D70770F48C010E94FD
:10F9F000C6FC8823E1F30E94B3FCF80181938F01D8
:10FA00002196CE15DF0598F381E090E0DF91CF914C
:10FA10001F910F91FF90EF90089590E0282F3327CA
:10FA20002138310589F02238310524F42038310598
:10FA300049F00DC02238310549F02839310539F433
:10FA400093E005C092E003C091E001C092E1892FEC
:10FA50009927089540E050E0609140017091410184
:10FA600046175707E8F4E2E4F1E0809142028EBBCA
:10FA70008091420290914302292F33272FBB019698
:10FA8000909343028093420280818DBBE29AE19A77
:10FA9000E199FECF4F5F5F4F31964617570728F326
:10FAA00008950F931F93CF93DF938091420290911B
:10FAB000430297FF03C081E08BBF01C01BBE00E083
:10FAC00010E0809140019091410108171907D8F486
:10FAD000C2E4D1E08091420290914302880F991FC5
:10FAE00060E0800F911F0E9480FC8883892F9927F6
:10FAF00089830E5F1F4F22968091400190914101B2
:10FB00000817190738F3DF91CF911F910F910895CE
:10FB100080914001909141010097C1F0E2E4F1E051
:10FB2000AC01809142028EBB8091420290914302CF
:10FB3000292F33272FBB01969093430280934202D3
:10FB4000E09A8DB381934150504059F708950F9337
:10FB50001F93CF93DF938C016115710541F0EB0189
:10FB6000F80181918F010E94D3FC2197C9F781E0B0
:10FB700090E0DF91CF911F910F9108950F931F9304
:10FB8000CF93DF93C0E0D0E00FEF11E0D0934302BA
:10FB9000C0934202D7FF03C081E08BBF01C01BBEF0
:10FBA000809142029091430263E0880F991F0E9466
:10FBB00065FC01501040C058DF4F17FFE7CF0E948F
:10FBC0009CFCDF91CF911F910F910895EF92FF92CE
:10FBD0000F931F93CF93DF93809142029091430242
:10FBE00097FF03C081E08BBF01C01BBE00E010E0A7
:10FBF00080914001909141010817190708F048C011
:10FC0000EE24FF24E801CD5BDE4FF801EE5BFE4FF2
:10FC1000EE0DFF1D4081888122969927382F2227DB
:10FC2000240F311D8091420290914302880F991F49
:10FC3000B9018E0D9F1D0E9470FC82E090E0E80EDD
:10FC4000F91E9FEFE916F10401F3F8F280914202E8
:10FC500090914302880F991F63E0800F911F0E94CB
:10FC600065FC8091420290914302880F991F65E0E4
:10FC7000800F911F0E9465FC0E949CFC00501F4F4A
:10FC800080914001909141010817190708F4B8CFFD
:10FC9000DF91CF911F910F91FF90EF900895CF9337
:10FCA000C0E069E081E090E00E9480FC84FF03C036
:10FCB0008F7E0E9493FC0E94C6FC8823E1F30E9481
:10FCC000B3FC992782359105DCF4803591050CF061
:10FCD00054C08134910509F45AC0823491053CF432
:10FCE0008033910509F449C0C19759F12FC182347D
:10FCF000910509F45FC08534910509F45EC026C101
:10FD00008635910509F4EDC0873591054CF48235AF
:10FD1000910509F461C08535910509F465C016C1E6
:10FD20008437910509F4A0C0853791052CF48436F9
:10FD3000910509F472C00AC18537910509F4C1C063
:10FD400005C10E94D8FC882309F4B5CF84E10E9444
:10FD5000D3FC81E40E94D3FC86E50E94D3FC82E5BB
:10FD60000E94D3FC80E20E94D3FC83E50E94D3FC76
:10FD700084E50E94D3FC8BE406C00E94D8FC882353
:10FD800009F499CF84E10E94D3FC80E1E0C061E0F6
:10FD900070E080E091E00E94EAFC0E94D8FC882399
:10FDA00009F489CF84E10E94D3FC809100010E9474
:10FDB0000DFDE9CF64E170E00AC061E070E080E031
:10FDC00091E00E94EAFC809100019927BC0180E04B
:10FDD00091E00E94EAFCD1CF0E94D8FC882309F46C
:10FDE0006ACF0E94BEFDCECF62E070E080E091E07D
:10FDF0000E94EAFC0E94D8FC882309F45CCF209181
:10FE00000001809101019927982F8827820F911D69
:10FE10009093430280934202B5CF63E070E080E0AC
:10FE200091E00E94EAFC2091010180910001992754
:10FE3000982F8827820F911D909341018093400154
:10FE4000BC0182E491E00E94EAFC0E94D8FC882375
:10FE500009F431CF80910201863419F40E94E6FD45
:10FE600091CF0E942AFD8ECF63E070E080E091E0A8
:10FE70000E94EAFC20910101809100019927982FAE
:10FE80008827820F911D90934101809340010E9429
:10FE9000D8FC882309F40FCF80910201863419F42D
:10FEA0000E9451FD02C00E9488FD84E10E94D3FCA3
:10FEB000609140017091410182E491E00E94A7FDB0
:10FEC00064CF0E94D8FC882309F4F5CE84E10E9417
:10FED000D3FC8EE10E94D3FC87E90E94D3FC82E030
:10FEE00052CF64E070E080E091E00E94EAFC0E9462
:10FEF000D8FC882309F4DFCE84E10E94D3FC8091F2
:10FF00000001803531F480910101882361F4C82F0C
:10FF100017C0883531F480910101883061F4C3E065
:10FF20000FC0803531F480910101883049F4C2E07E
:10FF300007C0883529F480910101882309F4C1E0C4
:10FF400069E08C2F99270E9480FC1DCF85E10E94DB
:10FF5000D3FCB1CECFEFD0E1DEBFCDBFCEE1F89480
:10FF60008EEF9FE00E94DDFF843B61F48FEF9FE006
:10FF70000E94DDFF833C31F48DEF9FE00E94DDFFA6
:10FF800080936F000E94AEFC0E94B3FC84E690E078
:10FF90000E94B6FC0E94C6FC882321F4C150C8BB55
:10FFA000CC23A1F7CC2319F00E944FFE02C00E947F
:10FFB000CEFC80E090E00C94E5FFE199FECF9FBB82
:0CFFC0008EBBE09A99278DB30895FFCF07
:040000031000F800F1
:00000001FF
